:020000040000FA
:020000002728AF
:080008002728820700000E34D6
:100010000D340A34093408340134A000A101A10BC5
:100020000F28A00B0E2808006530A200A301A30A28
:100030002308073C031916282308052086002208F8
:100040000D20A20A2208953C031D17280800F03055
:1000500083168600811383120F30860009308B00CF
:1000600086080B106300000086080B10A401A40A88
:100070002408073C031936282408052086000000C0
:10008000861F372814202408052086008030A5000C
:10009000FF300D20861F3628A50B48280F3086001C
:0200A000302806
:00000001FF
